** EXPERIMENTAL (HLL) ** Open Watcom Linker Version 1.6beta1 Limited Availability
Portions Copyright (c) 1985-2002 Sybase, Inc. All Rights Reserved.
Created on:       13/11/17 16:25:27
Warning! W1121: file U:/tmp\ldconv__curses_panel_obj_1a7f52885a4d17dfa0.obj(U:\DEV\python-2.7.5\Modules\_curses_panel.c): '_init_curses_panel' has already been exported
Executable Image: build/lib.os2knix-2.7/_curses_.pyd
creating an OS/2 EMX dynamic link library


                        +------------+
                        |   Groups   |
                        +------------+

Group                           Address              Size
=====                           =======              ====

CGROUP                          0001:00000000        0002a230
DGROUP                          0002:00000000        000012f0



                        +--------------+
                        |   Segments   |
                        +--------------+

Segment                Class          Group          Address         Size
=======                =====          =====          =======         ====

TEXT32                 CODE           CGROUP         0001:00000000   0002a230
________TEXT           CODE           CGROUP         0001:0002a230   00000000
DATA32                 DATA           DGROUP         0002:00000000   000009c0
SET1__os2dll           DATA           DGROUP         0002:000009c0   00000004
SET2__os2dll           DATA           DGROUP         0002:000009c4   00000000
SET3__os2dll           DATA           DGROUP         0002:000009c4   00000004
SET1___CTOR_LIST__     DATA           DGROUP         0002:000009c8   00000004
SET2___CTOR_LIST__     DATA           DGROUP         0002:000009cc   00000000
SET3___CTOR_LIST__     DATA           DGROUP         0002:000009cc   00000004
SET1___DTOR_LIST__     DATA           DGROUP         0002:000009d0   00000004
SET2___DTOR_LIST__     DATA           DGROUP         0002:000009d4   00000000
SET3___DTOR_LIST__     DATA           DGROUP         0002:000009d4   00000004
SET1___crtinit1__      DATA           DGROUP         0002:000009d8   00000004
SET2___crtinit1__      DATA           DGROUP         0002:000009dc   00000000
SET3___crtinit1__      DATA           DGROUP         0002:000009dc   00000004
SET1___crtexit1__      DATA           DGROUP         0002:000009e0   00000004
SET2___crtexit1__      DATA           DGROUP         0002:000009e4   00000000
SET3___crtexit1__      DATA           DGROUP         0002:000009e4   00000004
SET1___eh_frame__      DATA           DGROUP         0002:000009e8   00000004
SET2___eh_frame__      DATA           DGROUP         0002:000009ec   00000008
SET3___eh_frame__      DATA           DGROUP         0002:000009f4   00000004
SET1___eh_init__       DATA           DGROUP         0002:000009f8   00000004
SET2___eh_init__       DATA           DGROUP         0002:000009fc   00000004
SET3___eh_init__       DATA           DGROUP         0002:00000a00   00000004
SET1___eh_term__       DATA           DGROUP         0002:00000a04   00000004
SET2___eh_term__       DATA           DGROUP         0002:00000a08   00000004
SET3___eh_term__       DATA           DGROUP         0002:00000a0c   00000004
SET1___fork_parent1__  DATA           DGROUP         0002:00000a10   00000004
SET2___fork_parent1__  DATA           DGROUP         0002:00000a14   00000000
SET3___fork_parent1__  DATA           DGROUP         0002:00000a14   00000004
SET1___fork_child1__   DATA           DGROUP         0002:00000a18   00000004
SET2___fork_child1__   DATA           DGROUP         0002:00000a1c   00000000
SET3___fork_child1__   DATA           DGROUP         0002:00000a1c   00000004
________DATA           DATA           DGROUP         0002:00000a20   00000000
BSS32                  BSS            DGROUP         0002:00000a20   000008d0
c_common               BSS            DGROUP         0002:000012f0   00000000
________BSS            BSS            DGROUP         0002:000012f0   00000000


                        +----------------+
                        |   Memory Map   |
                        +----------------+

* = unreferenced symbol
+ = symbol only referenced locally

Address        Symbol
=======        ======

Module: U:\usr\lib\dll0hi.obj({standard input})
0001:00000000* __text
0002:00000000* __data
0002:00000000* ___data_start
0002:00000a20* ___bss_start
0002:000009c0+ __os2dll
0002:000009c8  ___CTOR_LIST__
0002:000009d0  ___DTOR_LIST__
0002:000009d8* ___crtinit1__
0002:000009e0* ___crtexit1__
0002:000009e8  ___eh_frame__
0002:000009f8  ___eh_init__
0002:00000a04  ___eh_term__
0002:00000a10+ ___fork_parent1__
0002:00000a18+ ___fork_child1__
Module: U:/tmp\ldconv__curses_panel_obj_1a7f52885a4d17dfa0.obj(U:\DEV\python-2.7.5\Modules\_curses_panel.c)
0001:0000095e  _init_curses_panel
0002:00000050* _PyCursesPanel_Type
Module: U:\usr\local473\lib\libc_dll.lib(dllinit.obj)
0001:00000ad0  _DLL_InitTerm
Module: U:\usr\lib\libend.lib(src/libend/386/endlink386.asm)
0002:000012f0  _end
0002:00000a20  _edata
Module: U:\usr\lib\libend.lib(src/libend/386/end.asm)
0001:0002a230* _etext
0001:0002a230* __etext
0000:00000000  WEAK$ZERO
0002:000012f0  __end
0002:00000a20  __edata
Module: U:\extras\lib\panel.lib(p_replace.obj)
0001:00000b30  _replace_panel
Module: U:\extras\lib\panel.lib(p_delete.obj)
0001:00000e40  _del_panel
Module: U:\extras\lib\panel.lib(p_update.obj)
0001:000011f0  _update_panels
Module: U:\extras\lib\panel.lib(p_user.obj)
0001:00001540  _set_panel_userptr
0001:00001560  _panel_userptr
Module: U:\extras\lib\panel.lib(p_move.obj)
0001:00001580  _move_panel
Module: U:\extras\lib\panel.lib(p_hidden.obj)
0001:000018b0  _panel_hidden
Module: U:\extras\lib\panel.lib(p_below.obj)
0001:00001900  _panel_below
Module: U:\extras\lib\panel.lib(p_above.obj)
0001:00001950  _panel_above
Module: U:\extras\lib\panel.lib(p_new.obj)
0001:000019a0  _new_panel
Module: U:\extras\lib\panel.lib(p_top.obj)
0001:00001ab0  _top_panel
Module: U:\extras\lib\panel.lib(p_show.obj)
0001:00001ac0  _show_panel
Module: U:\extras\lib\panel.lib(p_hide.obj)
0001:00001eb0  _hide_panel
Module: U:\extras\lib\panel.lib(p_bottom.obj)
0001:00002250  _bottom_panel
Module: U:\tmp\ldconv_libgcc_so_d_a_1a7f52885a4e15ff28.lib(emx-ctordtor.obj)
0001:00002660  ___ctordtorInit
0001:00002694  ___ctordtorTerm
Module: U:\extras\lib\ncurses.lib(lib_touch.obj)
0001:000026d0  _is_linetouched
0001:00002710* _is_wintouched
0001:00002750  _wtouchln
Module: U:\extras\lib\ncurses.lib(nc_panel.obj)
0001:00002810  __nc_panelhook
Module: U:\extras\lib\ncurses.lib(lib_refresh.obj)
0001:00002830  _wnoutrefresh
0001:00002a40  _wrefresh
Module: U:\extras\lib\ncurses.lib(lib_mvwin.obj)
0001:00002ab0  _mvwin
Module: U:\extras\lib\ncurses.lib(lib_data.obj)
0002:00000a60  _stdscr
0002:00000a64  _curscr
0002:00000a68  _newscr
0002:00000a6c  __nc_screen_chain
0002:00000a70  _SP
Module: U:\tmp\ldconv_libgcc_so_d_a_1a7f52885a4e15ff28.lib(emx-eh.obj)
0001:00002b50  ___ehInit
0001:00002b86* ___ehTerm
Module: U:\extras\lib\ncurses.lib(lib_window.obj)
0001:00002bc0* _wsyncup
0001:00002c90  _wsyncdown
0001:00002d70* _dupwin
0001:00002f80  __nc_synchook
0001:00002fc0* _mvderwin
0001:000030e0* _syncok
0001:00003100* _wcursyncup
Module: U:\extras\lib\ncurses.lib(tty_update.obj)
0001:00003170  _doupdate
0001:00005590* __nc_screen_resume
0001:00004ee0  __nc_scrolln
0001:00005730* __nc_screen_init
0001:00005740  __nc_screen_wrap
Module: U:\extras\lib\ncurses.lib(lib_pad.obj)
0001:00007960* _pnoutrefresh
0001:00007c80  _newpad
0001:00007d50* _subpad
0001:00007da0* _prefresh
0001:00007e00* _pechochar
Module: U:\extras\lib\ncurses.lib(lib_newwin.obj)
0001:00007e90  __nc_freewin
0001:00007f60  __nc_makenew
0001:000081b0  _newwin
0001:000082c0  _derwin
0001:00008400* _subwin
Module: U:\extras\lib\ncurses.lib(lib_move.obj)
0001:00008600  _wmove
Module: U:\extras\lib\ncurses.lib(lib_tstp.obj)
0001:00008650  __nc_signal_handler
Module: U:\extras\lib\ncurses.lib(lib_vidattr.obj)
0001:00008af0* _vidputs
0001:000093f0  _vidattr
0001:00009410  _termattrs
Module: U:\extras\lib\ncurses.lib(lib_tputs.obj)
0001:00009920  __nc_outch
0001:000094c0  _tputs
0001:00009820* _delay_output
0001:000098f0  __nc_flush
0001:00009980  _putp
0002:00000af0  _PC
0002:00000af2  _ospeed
0002:00000af4* __nc_nulls_sent
Module: U:\extras\lib\ncurses.lib(lib_mvcur.obj)
0001:000099c0* __nc_msec_cost
0001:00009b40* __nc_mvcur_init
0001:0000a520  _mvcur
0001:0000a710  __nc_mvcur_resume
0001:0000a7c0  __nc_mvcur_wrap
Module: U:\extras\lib\ncurses.lib(hardscroll.obj)
0001:0000b670  __nc_scroll_optimize
0002:00000b00  __nc_oldnums
Module: U:\extras\lib\ncurses.lib(lib_ttyflags.obj)
0001:0000b840* __nc_get_tty_mode
0001:0000b8c0  __nc_set_tty_mode
0001:0000b940  _def_shell_mode
0001:0000b9c0  _def_prog_mode
0001:0000ba40  _reset_prog_mode
0001:0000baf0  _reset_shell_mode
0001:0000bbc0* _savetty
0001:0000bc40* _resetty
Module: U:\extras\lib\ncurses.lib(lib_cur_term.obj)
0001:0000bcc0  _set_curterm
0001:0000bd20  _del_curterm
0002:00000b50  _cur_term
Module: U:\extras\lib\ncurses.lib(lib_color.obj)
0001:0000bec0* _start_color
0001:0000c150* _init_pair
0001:0000c460  __nc_do_color
0001:0000c7e0  __nc_reset_colors
0001:0000c870  _init_color
0001:0000cb50* _can_change_color
0001:0000cb70  _has_colors
0001:0000cbf0* _color_content
0001:0000cc90  _pair_content
0002:00000b60  _COLOR_PAIRS
0002:00000b64  _COLORS
Module: U:\extras\lib\ncurses.lib(lib_has_cap.obj)
0001:0000ce60  _has_ic
0001:0000ced0  _has_il
Module: U:\extras\lib\ncurses.lib(lib_tparm.obj)
0001:0000cf30* __nc_tparm_analyze
0001:0000d260  _tparm
0002:00000b70* __nc_tparm_err
Module: U:\extras\lib\ncurses.lib(lib_scroll.obj)
0001:0000e400  __nc_scroll_window
0001:0000e660  _wscrl
Module: U:\extras\lib\ncurses.lib(hashmap.obj)
0001:0000e6d0  __nc_hash_map
0001:0000ec00  __nc_make_oldhash
0001:0000ec60  __nc_scroll_oldhash
Module: U:\extras\lib\ncurses.lib(lib_addch.obj)
0001:0000f5f0  __nc_render
0001:0000f6b0  __nc_waddch_nosync
0001:0000f6c0  _waddch
0001:0000f710  _wechochar
Module: U:\extras\lib\ncurses.lib(lib_endwin.obj)
0001:0000ff10  _endwin
Module: U:\extras\lib\ncurses.lib(lib_kernel.obj)
0001:0000ff50* _erasechar
0001:0000ff80* _killchar
0001:0000ffb0  _flushinp
Module: U:\extras\lib\ncurses.lib(lib_set_term.obj)
0001:00010010* _delscreen
0001:00010310* __nc_setupscreen
0001:000109b0* __nc_ripoffline
0001:000109f0  _set_term
0001:00010a60* _ripoffline
Module: U:\extras\lib\ncurses.lib(lib_napms.obj)
0001:00010b20  _napms
Module: U:\extras\lib\ncurses.lib(lib_baudrate.obj)
0001:00010c10  __nc_baudrate
0001:00010c60  __nc_ospeed
0001:00010ca0  _baudrate
Module: U:\extras\lib\ncurses.lib(lib_options.obj)
0001:00010cf0  _curs_set
0001:00010db0* _idlok
0001:00010e10* _idcok
0001:00010e60* _halfdelay
0001:00010eb0* _nodelay
0001:00010ee0* _notimeout
0001:00010f00* _wtimeout
0001:00010f20* _keypad
0001:00010fb0* _meta
0001:00011020* _typeahead
0001:00011040* _has_key
0001:000110c0  __nc_keypad
Module: U:\extras\lib\ncurses.lib(strings.obj)
0001:000111b0  __nc_str_init
0001:000111e0  __nc_str_null
0001:00011210  __nc_str_copy
0001:00011240  __nc_safe_strcat
0001:000112b0  __nc_safe_strcpy
Module: U:\extras\lib\ncurses.lib(doalloc.obj)
0001:00011320  __nc_doalloc
Module: U:\extras\lib\ncurses.lib(setbuf.obj)
0001:000113a0  __nc_set_buffer
Module: U:\extras\lib\ncurses.lib(free_ttype.obj)
0001:00011460  __nc_free_termtype
0001:00011520* _use_extended_names
0002:00000360  __nc_user_definable
Module: U:\extras\lib\ncurses.lib(comp_error.obj)
0001:00011570  __nc_warning
0001:00011680  __nc_err_abort
0001:00011790  __nc_syserr_abort
0001:000118a0* __nc_get_source
0001:000118b0* __nc_set_source
0001:000118c0  __nc_set_type
0001:00011920  __nc_get_type
0002:00000dc0  __nc_suppress_warnings
0002:00000dc4  __nc_curr_line
0002:00000dc8  __nc_curr_col
Module: U:\extras\lib\ncurses.lib(unctrl.obj)
0001:00012070  _unctrl
Module: U:\extras\lib\ncurses.lib(lib_clreol.obj)
0001:000120d0  _wclrtoeol
Module: U:\extras\lib\ncurses.lib(lib_setup.obj)
0001:00012330* __nc_setupterm
0001:000127d0* _use_env
0001:000127e0* __nc_get_locale
0001:00012810  __nc_unicode_locale
0001:00012880  __nc_locale_breaks_acs
0001:000129e0* _setupterm
0002:00000370* _ttytype
0002:00000df0  _LINES
0002:00000df4  _COLS
0002:00000df8  _TABSIZE
Module: U:\extras\lib\ncurses.lib(lib_slk.obj)
0001:00012b50  __nc_slk_initialize
0001:000130e0* _slk_restore
0002:00000e00* __nc_slk_format
Module: U:\extras\lib\ncurses.lib(lib_acs.obj)
0001:00013200  __nc_init_acs
0002:00000e10  _acs_map
Module: U:\extras\lib\ncurses.lib(lib_raw.obj)
0001:00013580* _raw
0001:00013640  _cbreak
0001:000136f0* _qiflush
0001:00013750* _noraw
0001:00013810* _nocbreak
0001:000138b0* _noqiflush
0001:00013910* _intrflush
Module: U:\extras\lib\ncurses.lib(init_keytry.obj)
0001:00013990  __nc_init_keytry
0002:00000490* __nc_tinfo_fkeys
Module: U:\extras\lib\ncurses.lib(comp_parse.obj)
0001:00013ad0* __nc_delink_entry
0001:00013b80* __nc_read_entry_source
0001:00013d70* __nc_resolve_uses2
0001:00015670* __nc_free_entries
0001:000156a0  __nc_free_entry
0001:000156d0* __nc_entry_match
0001:00015870* __nc_resolve_uses
0002:00000950* __nc_check_termtype2
0002:00000954* __nc_check_termtype
0002:00001010  __nc_head
0002:00001014* __nc_tail
Module: U:\extras\lib\ncurses.lib(read_entry.obj)
0001:000158b0* __nc_read_termtype
0001:00016310* __nc_read_file_entry
0001:000163c0  __nc_read_entry
Module: U:\extras\lib\ncurses.lib(fallback.obj)
0001:00016690  __nc_fallback
Module: U:\extras\lib\ncurses.lib(name_match.obj)
0001:000166a0  __nc_name_match
0001:00016790  __nc_first_name
Module: U:\extras\lib\ncurses.lib(getenv_num.obj)
0001:00016800  __nc_getenv_num
Module: U:\extras\lib\ncurses.lib(lib_hline.obj)
0001:00016860  _whline
Module: U:\extras\lib\ncurses.lib(lib_printw.obj)
0001:00016920* _printw
0001:00016a20* _vwprintw
0001:00016950* _wprintw
0001:00016980* _mvprintw
0001:000169d0  _mvwprintw
Module: U:\extras\lib\ncurses.lib(lib_slkrefr.obj)
0001:00016a70* _slk_noutrefresh
0001:00016ad0  _slk_refresh
Module: U:\extras\lib\ncurses.lib(key_defined.obj)
0001:00016d90  _key_defined
Module: U:\extras\lib\ncurses.lib(add_tries.obj)
0001:00016dd0  __nc_add_to_try
Module: U:\extras\lib\ncurses.lib(names.obj)
0001:00017020* _boolnames
0001:000173c0  _boolfnames
0001:00017540* _numnames
0001:00017840  _numfnames
0001:000180c0  _strnames
0001:00019b00  _strfnames
Module: U:\extras\lib\ncurses.lib(comp_scan.obj)
0001:0001a410  __nc_get_token
0001:0001b210  __nc_panic_mode
0001:0001ad30* __nc_trans_string
0001:0001b230  __nc_reset_input
0001:0001b290  __nc_push_token
0002:00001040  __nc_syntax
0002:00001044* __nc_curr_file_pos
0002:00001048  __nc_comment_start
0002:0000104c  __nc_comment_end
0002:00001050  __nc_start_line
0002:00001054  __nc_curr_token
0002:00001060* __nc_disable_period
Module: U:\extras\lib\ncurses.lib(parse_entry.obj)
0001:0001bf80  __nc_parse_entry
0001:0001c710* __nc_capcmp
Module: U:\extras\lib\ncurses.lib(alloc_entry.obj)
0001:0001def0  __nc_wrap_entry
0001:0001e460  __nc_merge_entry
0001:0001e560  __nc_init_entry
0001:0001e680  __nc_copy_entry
0001:0001e6f0  __nc_save_str
Module: U:\extras\lib\ncurses.lib(alloc_ttype.obj)
0001:0001e790  __nc_align_termtype
0001:0001ea70  __nc_copy_termtype
Module: U:\tmp\ldconv_libgcc_a_1a7f52885a4d18c230.lib(_alloca.obj)
0001:0001f730  __alloca
Module: U:\extras\lib\ncurses.lib(access.obj)
0001:0001f770* __nc_rootname
0001:0001f810* __nc_is_abs_path
0001:0001f850  __nc_pathlast
0001:0001f8a0* __nc_basename
0001:0001f8f0  __nc_access
0001:0001f9c0  __nc_is_dir_path
0001:0001fa10* __nc_is_file_path
Module: U:\extras\lib\ncurses.lib(db_iterator.obj)
0001:0001fab0  __nc_next_db
0001:0001fbf0* __nc_tic_dir
0001:0001fc40* __nc_keep_tic_dir
0001:0001fc90  __nc_last_db
0001:0001fcd0* __nc_first_db
Module: U:\extras\lib\ncurses.lib(safe_sprintf.obj)
0001:0001fdc0  __nc_printf_string
Module: U:\extras\lib\ncurses.lib(lib_addstr.obj)
0001:0001fed0* _waddchnstr
0001:0001ffe0  _waddnstr
Module: U:\extras\lib\ncurses.lib(lib_trace.obj)
0002:000011e0  __nc_tracing
Module: U:\extras\lib\ncurses.lib(comp_captab.obj)
0001:00022130  __nc_info_hash_table
0001:00024d70  __nc_cap_hash_table
0001:00025d90  __nc_capalias_table
0001:00025fd0  __nc_infoalias_table
0001:00026030  __nc_get_table
0001:00026050* __nc_get_hash_table
Module: U:\extras\lib\ncurses.lib(comp_hash.obj)
0001:00026070  __nc_find_entry
0001:00026110  __nc_find_type_entry
Module: U:\extras\lib\ncurses.lib(captoinfo.obj)
0001:00026250  __nc_captoinfo
0001:00027500* __nc_infotocap
Module: U:\extras\lib\ncurses.lib(visbuf.obj)
0001:00029ef0* __nc_visbuf2
0001:00029f90  __nc_visbuf
0001:00029fb0* __nc_visbufn
Module: U:\extras\lib\ncurses.lib(home_terminfo.obj)
0001:0002a1a0  __nc_home_terminfo


                        +----------------------+
                        |   Imported Symbols   |
                        +----------------------+

Symbol                              Module
======                              ======

___libc_ForkRegisterModule          libc065
___init_dll                         libc065
___libc_Back_termDll                libc065
___libc_ForkDeregisterModule        libc065
__atfork_callback                   libc065
_Py_FindMethod                      python27
_PyTuple_Size                       python27
_PyArg_ParseTuple                   python27
_PyExc_RuntimeError                 python27
_PyErr_SetString                    python27
_PyExc_TypeError                    python27
__Py_NoneStruct                     python27
_PyObject_Free                      python27
_PyErr_Format                       python27
__Py_TrueStruct                     python27
__Py_ZeroStruct                     python27
_PyObject_Malloc                    python27
_PyObject_Init                      python27
_PyErr_NoMemory                     python27
_PyType_Type                        python27
_PyCapsule_Import                   python27
_Py_InitModule4                     python27
_PyModule_GetDict                   python27
_PyErr_NewException                 python27
_PyDict_SetItemString               python27
_PyString_FromString                python27
__CRT_init                          libc065
__CRT_term                          libc065
__std_free                          libc065
__std_malloc                        libc065
___ctordtorInit1                    libc065
___ctordtorTerm1                    libc065
__std_fwrite                        libc065
___register_frame_table             gcc473
___deregister_frame                 gcc473
___libc_GLocaleCtype                libc065
___stdoutp                          libc065
__std_select                        libc065
__errno                             libc065
__std_putc                          libc065
__std_calloc                        libc065
__std_sigaction                     libc065
__std_sigemptyset                   libc065
__std_sigaddset                     libc065
__std_sigprocmask                   libc065
__std_sigismember                   libc065
__std_getpid                        libc065
__std_kill                          libc065
__std_tcgetpgrp                     libc065
__std_getpgrp                       libc065
__std_exit                          libc065
__std_fileno                        libc065
__std_isatty                        libc065
__std_strchr                        libc065
__std_fflush                        libc065
__std_write                         libc065
__std_strstr                        libc065
__std_strlen                        libc065
__std_tcgetattr                     libc065
__std_tcsetattr                     libc065
__std_sprintf                       libc065
___stderrp                          libc065
__std_memmove                       libc065
__scrsize                           libc065
__std_tcflush                       libc065
__std_getenv                        libc065
__std_sscanf                        libc065
__std_nanosleep                     libc065
__std_cfgetospeed                   libc065
__std_strcpy                        libc065
__std_realloc                       libc065
__std_setvbuf                       libc065
__std_fprintf                       libc065
__std_fputc                         libc065
__std_vfprintf                      libc065
__std_strncat                       libc065
__std_strncpy                       libc065
__std_strdup                        libc065
__std_strcmp                        libc065
__std_setlocale                     libc065
__std_nl_langinfo                   libc065
__std_atoi                          libc065
__std_memset                        libc065
__std_setmode                       libc065
__std_memcpy                        libc065
__std_open                          libc065
__std_read                          libc065
__std_close                         libc065
__std_strtol                        libc065
__std_ftell                         libc065
__std_fgets                         libc065
__std_strcat                        libc065
__std_strncmp                       libc065
__std_strrchr                       libc065
__std_access                        libc065
__std_stat                          libc065
__std_vsnprintf                     libc065


                        +--------------------+
                        |   Libraries Used   |
                        +--------------------+

U:\extras\lib\panel.lib
U:\extras\lib\ncurses.lib
U:\tmp\ldconv_python2_7_dll_a_1a7f52885a4d188798.lib
U:\tmp\ldconv_libgcc_a_1a7f52885a4d18c230.lib
U:\tmp\ldconv_libgcc_so_d_a_1a7f52885a4e15ff28.lib
U:\usr\lib\libc_alias.lib
U:\usr\local473\lib\libc_dll.lib
U:\usr\lib\libend.lib


                        +-----------------------+
                        |   Linker Statistics   |
                        +-----------------------+

Stack size:  0000 (0.)
Memory size:  0002b520 (177440.)
Link time: 00:00.12
